:1000000012C02BC02AC029C028C027C096C0B8C0C3
:10001000DAC088C022C021C020C01FC0EDC01DC0F2
:100020001CC01BC01AC011241FBECFE5D4E0DEBF28
:10003000CDBF10E0A0E6B0E0ECE3F2E002C0059036
:100040000D92A036B107D9F710E0A0E6B0E001C0EC
:100050001D92A236B107E1F743C0D2CFA99B02C0DF
:10006000A9980895A99A08950895A89B02C0A898F0
:100070000895A89A0895089581B3806381BB82B3DF
:10008000806382BB87B3806387BB88B3806388BB90
:1000900087B3866087BB88B3897F88BB08958EB598
:1000A000827382618EBD8FB582E08FBD89B78E71FC
:1000B0008C6189BF08958FB780688FBF089587B11D
:1000C0008077806687B986B18EE886B9089583B750
:1000D0008D7F856083BF89B7816089BF12BE089517
:1000E000CFE5D4E0DEBFCDBF85B5887F85BDC098A4
:1000F000B89A92988A9A96988E9A97988F9A85B37A
:100100008C7F85BB84B3836084BBB6DFC8DF17BC3C
:100110008FEF86BDD0DFD3DF87B1837F836087B960
:10012000D6DFFFCF1F920F920FB60F921124369A8F
:100130000F900FBE0F901F9018951F920F920FB641
:100140000F9211242F933F934F935F936F937F935D
:100150008F939F93AF93BF93EF93FF937FDFFF91B5
:10016000EF91BF91AF919F918F917F916F915F912F
:100170004F913F912F910F900FBE0F901F901895A8
:100180001F920F920FB60F9211242F933F934F930C
:100190005F936F937F938F939F93AF93BF93EF93EF
:1001A000FF9363DFFF91EF91BF91AF919F918F918B
:1001B0007F916F915F914F913F912F910F900FBE63
:1001C0000F901F9018951F920F920FB60F92112447
:1001D0008F939F9380916000809599279BBD8ABDE6
:1001E00080916100992799BD88BD9F918F910F9053
:1001F0000FBE0F901F9018951F920F920FB60F927F
:1002000011248F939F9387B199278F7090700397D4
:1002100039F485B18093600087B1827F826006C027
:1002200085B18093610087B1837F836087B99F9197
:0C0230008F910F900FBE0F901F9018953B
:00000001FF
